:020000020000FC
:100000000FC0A0C0C3C0C3C0C3C0C3C0C3C0C3C0AF
:02001000C3C06B
:10002000F89411E00EE51EBF0DBF00E811E006BD1B
:1000300016BD00E00BBF00E009BF00E005BB00E615
:100040000ABF06E408BF04E208BB0BE107BB01E0FE
:1000500005BF03E000BD00E00ABD03E003BF00E010
:1000600009BD00E008BD00E000BF00E00CBD00E0FD
:100070000EBD00E00BBD0CE00DBD00E007BD09E8C2
:1000800000BF00E007B900E003B900E006B900E0F6
:1000900004BB00E808B9A89504B7077F04BF01B501
:1000A000006101BD0DE401BD00E40BBF00E009BF2C
:1000B00091E00DE5102E00E0C02E7894A8950BE19C
:1000C00007BBC03021F0CA9479F4CA950DC0C0981E
:1000D000C39800B70F7800BFC1980CB50F780CBD5E
:1000E000C0980DE5102EEACF212D213518F02A36C3
:1000F00078F41CC000B70F7800BFC198C098C39AAD
:100100000CB5037800660CBD11E5121B1BBD19C0B0
:100110000CB503780CBDC498C398C09A00B70F788B
:10012000006E00BF1AE6211B2EBD0BC000B70F7872
:1001300000BF0CB503780CBDC198C498C098C39893
:1001400000C0BCCFFFB646B342FF18C0512D42B726
:100150004F31D0F04C39C0F4451779F038F4541BC6
:1001600061E05A3008F062E0161A07C0451B61E0F2
:10017000AA3008F062E0160E00C006C04CB541601F
:100180004CBD442742BFC2E3FFBE18951895189591
:0A0190001895189518951895189504
:00000001FF
